:020000040000FA
:06000000C93001303A286E
:08000800A000030EA100831209
:1000100005191028831601178312B23081002B288E
:1000200083160113831203140B190310A80DA90DD5
:10003000AA0DAB0DAC0DAC16FF302C02031D2B2806
:10004000FA302B02031D2B2831152A08AF0029088E
:10005000AE002808AD008B100B11210E8300A00EFE
:04006000200E090065
:0C007400203084008001840A80300402E7
:10008000031C3C281230B000E02183160C3085059B
:1000900087018312850187010730990000309A009B
:1000A000103083168E008312603083168F00831207
:1000B0000030831691009F008312C83083168100A0
:1000C000831231309000003083168C008312103080
:1000D0008B00831600309B001C141A088312BC008E
:1000E000851DD222831610309B001C141A0883121F
:1000F000BD00831630309B001C141A088312DE00EA
:10010000B92281018E018F010B118B100B108C0114
:100110008B17982031199B20B30B96280310851953
:100120000314B90DF030390203194421182389282A
:1001300064003210080031110130B7008B132030F9
:10014000370783169B001C141A088312A400103072
:10015000370783169B001C141A088312A300A600FD
:100160000230A6060030370783169B001C141A08BD
:100170008312A200A7000130A7068B17321CC628E5
:1001800022090339A200A309A409A50924082F0202
:10019000031D3E2923082E02031D3E2922082D029D
:1001A000031D3E2901303702031DDB283D18DB28E3
:1001B0003D143E14ED2102303702031DE428BD1822
:1001C000E428BD143E14FC2103303702031DED2842
:1001D0003D19ED283D153E14082204303702031D59
:1001E000F628BD19F628BD153E1414220530370235
:1001F000031DFF283D1AFF283D163E14232206301A
:100200003702031D0829BD1A0829BD163E142F22E6
:1002100007303702031D11293D1B11293D173E14DC
:100220003B2208303702031D1A29BD1B1A29BD17AE
:100230003E14462209303702031D23295E18232964
:100240005E143E1451220A303702031D2C29DE1899
:100250002C29DE143E145C220B303702031D352995
:100260005E1935295E153E1467220C303702031DD6
:100270003E29DE193E29DE153E147222B70A0D30E2
:100280003702031808009E280130B600B300B400FE
:10029000B500B70085018701B1139820B30B8C29F5
:1002A000031085190314B90DF03039020319B3296D
:1002B000B40B8C290130370203197D22023037023A
:1002C00003198222033037020319872204303702D0
:1002D00003198C22053037020319912206303702A8
:1002E000031996220730370203199B220830370280
:1002F0000319A022093037020319A5220A30370258
:100300000319AA220B3037020319AF220C3037022F
:100310000319B4229630B400311D4D293111321C1D
:1003200096292D090339AD00AE09AF092F1C4D29BF
:100330008E018F010C1C4D290C102E1E4D298B1384
:1003400020303707BB002F08BA00CB211030370709
:10035000BB002E08BA00CB2100303707BB002D08A8
:10036000BA00CB218B1785018701B70AB6010D3082
:100370003702031C4D29B92208003E1C08003E101C
:100380001030BB003D08BA00CB213030BB005E0806
:10039000BA00CB2108008B133A0883161C159A006B
:1003A00083123B0883169B0055309D00AA309D00A8
:1003B0009C1464009C18D9291C1183128B17080007
:1003C000FF30C800CA15CB15CC15CD15CE15CF15ED
:1003D000D015D115D215D3150800C130BD05FF3099
:1003E000DE050130C405C0000030C200C600BC18E4
:1003F0005F14BC18DF140800C230BD05FF30DE05F5
:100400000230C405C0000030C200C6005F10080002
:10041000C430BD05FF30DE050630C405C000003025
:10042000C200C6005F100800C830BD05FF30DE0501
:100430001830C405C0000030C200C600BC185F14EC
:10044000BC18DF140800D030BD05FF30DE052230B7
:10045000C405C0000030C200C6005F100800E030D4
:10046000BD05FF30DE052630C405C0000030C200E7
:10047000C6005F1008007F30BD05C030DE05C0300B
:10048000C505C1000030C300C7000800BF30BD056E
:10049000C030DE053030C505C1000030C300C700E4
:1004A00008003F30BD05C130DE059030C505C100F4
:1004B0000030C300C70008003F30BD05C230DE0574
:1004C000C030C505C1000030C300C70008003F3080
:1004D000BD05C430DE053030C505C1000030C300A5
:1004E000C70008003F30BD05C830DE059030C505A7
:1004F000C1000030C300C70008001030850600307E
:100500008706080020308506003087060800213065
:10051000850600308706080002308506023087060F
:100520000800203085060430870608002130850643
:10053000043087060800003085061830870608005A
:100540000030850621308706080000308506093016
:10055000870608000030850618308706080000303E
:100560008506213087060800003085060930870699
:1005700008003D18ED21BD18FC213D190822BD19C8
:1005800014223D1A2322BD1A2F223D1B3B22BD1BE4
:1005900046225E185122DE185C225E196722DE199F
:1005A00072220800B601B301B4013C1CDA2ABC0176
:1005B000BC14DC2ABC013C143C08B6006400E02AF0
:1005C000E12AE22AE32AE42AFF30B41B8500B41FA3
:1005D0008501B30BDE2AB40BDE2A0310B60CB60875
:1005E000031DDE2A0030BB003C08BA00CB21080006
:1005F00005125C180516DC1C8512DC1885165C1DBE
:1006000005105C190514DC1D8510DC1985145C1EB1
:1006100087105C1A8714DC1E0711DC1A07155C1F93
:1006200007105C1B0714DC1F8712DC1B87160800F1
:100630008F08031908008F0178308E00C80F4A2DEB
:10064000C80A441C482B461C392BCA1C2A2BCA0139
:100650004A15562B4A1D2F2BCA01CA15562BCA1DE7
:10066000342BCA014A16562B4A1E562BCA01CA14ED
:10067000562B4A1D3E2BCA014A16562BCA1D432B28
:10068000CA014A16562B4A1E562BCA01CA14562BAB
:10069000CA1C4D2BCA014A15562B4A1D522BCA01A2
:1006A000CA15562B4A1E562BCA014A15C41C7D2B4F
:1006B000C61C6E2BCB1C5F2BCB014B158B2B4B1D04
:1006C000642BCB01CB158B2BCB1D692BCB014B1690
:1006D0008B2B4B1E8B2BCB01CB148B2B4B1D732BDE
:1006E000CB014B168B2BCB1D782BCB014B168B2BB9
:1006F0004B1E8B2BCB01CB148B2BCB1C822BCB011A
:100700004B158B2B4B1D872BCB01CB158B2B4B1EEE
:100710008B2BCB014B15441DB22B461DA32BCC1CA0
:10072000942BCC014C15C02B4C1D992BCC01CC1516
:10073000C02BCC1D9E2BCC014C16C02B4C1EC02BAD
:10074000CC01CC14C02B4C1DA82BCC014C16C02BBB
:10075000CC1DAD2BCC014C16C02B4C1EC02BCC019C
:10076000CC14C02BCC1CB72BCC014C15C02B4C1D72
:10077000BC2BCC01CC15C02B4C1EC02BCC014C1576
:10078000C41DE82BC61DD92BCD1CCA2BCD014D1580
:100790005F13F62B4D1DCF2BCD01CD15F62BCD1DA7
:1007A000D42BCD014D16F62B4D1EF62BCD01CD14BD
:1007B000F62B4D1DDE2BCD014D16F62BCD1DE32B5B
:1007C000CD014D16F62B4D1EF62BCD01CD14F62B7B
:1007D000CD1CED2BCD014D15F62B4D1DF22BCD0172
:1007E000CD15F62B4D1EF62BCD014D155F1B1F2C85
:1007F000441E1F2C461E102CCE1C012CCE014E1563
:100800002D2C4E1D062CCE01CE152D2CCE1D0B2CC5
:10081000CE014E162D2C4E1E2D2CCE01CE142D2C7D
:100820004E1D152CCE014E162D2CCE1D1A2CCE0190
:100830004E162D2C4E1E2D2CCE01CE142D2CCE1C42
:10084000242CCE014E152D2C4E1D292CCE01CE155B
:100850002D2C4E1E2D2CCE014E15C41E542CC61E02
:10086000452CCF1C362CCF014F15622C4F1D3B2C35
:10087000CF01CF15622CCF1D402CCF014F16622C1B
:100880004F1E622CCF01CF14622C4F1D4A2CCF017A
:100890004F16622CCF1D4F2CCF014F16622C4F1ECE
:1008A000622CCF01CF14622CCF1C592CCF014F15D5
:1008B000622C4F1D5E2CCF01CF15622C4F1E622C77
:1008C000CF014F15DF188B2C451E8B2C471E7C2C1F
:1008D000D01C6D2CD0015015992C501D722CD001BC
:1008E000D015992CD01D772CD0015016992C501E64
:1008F000992CD001D014992C501D812CD001501668
:10090000992CD01D862CD0015016992C501E992C54
:10091000D001D014992CD01C902CD0015015992CBA
:10092000501D952CD001D015992C501E992CD0011A
:100930005015DF18C22CC51EC22CC71EB32CD11CEB
:10094000A42CD1015115D02C511DA92CD101D115A8
:10095000D02CD11DAE2CD1015116D02C511ED02C33
:10096000D101D114D02C511DB82CD1015116D02C4D
:10097000D11DBD2CD1015116D02C511ED02CD1012E
:10098000D114D02CD11CC72CD1015115D02C511D04
:10099000CC2CD101D115D02C511ED02CD101511508
:1009A000DF18FA2C451FFA2C471FEB2CD21CDC2C2D
:1009B000D2015215DF13082D521DE12CD201D215A0
:1009C000082DD21DE62CD2015216082D521E082DDC
:1009D000D201D214082D521DF02CD2015216082D2E
:1009E000D21DF52CD2015216082D521E082DD2010F
:1009F000D214082DD21CFF2CD2015215082D521DE5
:100A0000042DD201D215082D521E082DD2015215E7
:100A1000DF18332DDF1B332DC51F332DC71F242DAA
:100A2000D31C152DD3015315412D531D1A2DD30160
:100A3000D315412DD31D1F2DD3015316412D531E08
:100A4000412DD301D314412D531D292DD30153160C
:100A5000412DD31D2E2DD3015316412D531E412D53
:100A6000D301D314412DD31C382DD3015315412D5F
:100A7000531D3D2DD301D315412D531E412DD301BF
:100A80005315BD214008C4004108C5005F18DF149C
:100A90005F1CDF104808C9000C304A05031D051211
:100AA0000C304B05031D85120C304C05031D051041
:100AB0000C304D05031D85100C304E05031D8710AD
:100AC0000C304F05031D07110C305005031D071096
:100AD0000C305105031D87120C305205031D0712FF
:100AE0000C305305031D871149080E020318A42D6D
:100AF00012304A05031D051612304B05031D8516DD
:100B000012304C05031D051412304D05031D8514CC
:100B100012304E05031D871412304F05031D0715B3
:100B200012305005031D071412305105031D87169E
:100B300012305205031D071612305305031D871589
:100B4000FF304802031908008F08031D0800982091
:100B500049080E02031CA42D18304A05031D051276
:100B600006304A05031D051618304B05031D851276
:100B700006304B05031D851618304C05031D051066
:100B800006304C05031D051418304D05031D851056
:100B900006304D05031D851418304E05031D8710C2
:100BA00006304E05031D871418304F05031D07112D
:100BB00006304F05031D071518305005031D07109B
:100BC00006305005031D071418305105031D871208
:100BD00006305105031D871618305205031D0712F4
:100BE00006305205031D071618305305031D8711E3
:0A0BF00006305305031D87150800A9
:084000000100030003000700AA
:02400E00CC33B1
:10420000010078007A007C007E007B0079007F004E
:104210007D007A0078007E007C007D007F00FF003A
:104220000200F200F600FA00FE00F200F600FA00CA
:10423000FE00F200F600FA00FE00F200F600FF00B9
:10424000FF00050005000500050009000900090040
:1042500009000D000D000D000D0011001100FF0000
:104260000100FF00FF00FF00FF00FF00FF00FF0054
:10427000FF00FF00FF00FF00FF00FF00FF00FF0046
:10428000FF00FF00FF00FF00FF00FF00FF00FF0036
:10429000FF00FF00FF00FF00FF00FF00FF00FF0026
:1042A000FF00FF00FF00FF00FF00FF00FF00FF0016
:1042B000FF00FF00FF00FF00FF00FF00FF00FF0006
:1042C000FF00FF00FF00FF00FF00FF00FF00FF00F6
:1042D000FF00FF00FF00FF00FF00FF00FF00FF00E6
:1042E000FF00FF00FF00FF00FF00FF00FF00FF00D6
:1042F000FF00FF00FF00FF00FF00FF00FF00DD00E8
:00000001FF
